:1000000009C021C020C01FC01EC01DC01CC01BC015
:100010008AC119C011241FBECFE9CDBF10E0A0E6F0
:10002000B0E0E8EBF3E002C005900D92AC36B1070A
:10003000D9F710E0ACE6B0E001C01D92AE36B107D2
:10004000E1F746D1B7C1DCCF87708064F894A895FA
:1000500098E191BD81BD7894089567B398B3B99A3A
:10006000C19848E750E013C0C19A20ED37E0FA018B
:100070003197F1F721503040D1F7C19820ED37E0AA
:10008000FA013197F1F721503040D1F781508823A0
:1000900059F767BB98BB089520E048E750E011C0CE
:1000A000C19A80ED97E0FA013197F1F70197D9F7FE
:1000B000C19880ED97E0FA013197F1F70197D9F7F0
:1000C0002F5F233068F380EA9FE0FA013197F1F760
:1000D0000197D9F720E0C19A80E797E1FA013197BB
:1000E000F1F70197D9F7C19880ED97E0FA013197C0
:1000F000F1F70197D9F72F5F233069F780EA9FE086
:10010000FA013197F1F70197D9F720E0C19A80ED14
:1001100097E0FA013197F1F70197D9F7C19880ED8F
:1001200097E0FA013197F1F70197D9F72F5F233064
:1001300069F780E593ECFA013197F1F70197D9F768
:1001400020E0AECF40E068E770E018C0C19A80EDD3
:1001500097E0FB013197F1F70197D9F7C1982AE0B1
:1001600030E008C0FB013197F1F70197D9F7215032
:10017000304019F080E197E2F5CF4F5F463030F321
:100180000AC0FB013197F1F70197D9F721503040B0
:1001900021F440E0DBCF22E330E080E197E2F1CFD1
:1001A000EF92FF920F931F93082F000F000F10E0A4
:1001B000C8014996E9D0F82EC8014A96E5D0E82E44
:1001C000C8014B96E1D0382FB99AC19881E28FBD12
:1001D00081E083BF80E040EB54E00EC0282F2E0D5D
:1001E000281708F42F2D29BD8AE090E0FA013197F5
:1001F000F1F70197D9F7822F8F1580F30EC0282FC2
:10020000231B821708F420E029BD8AE090E0FA0160
:100210003197F1F70197D9F7822F882381F720E0F2
:10022000EACFEF92FF920F931F93CF93DF93880F44
:10023000880FC82FD0E0CE014996A6D0082FCE0156
:100240004A96A2D0E82ECE014B969ED010E0B8017F
:10025000660F771F20E0F02E012FA0EBB4E0482FAF
:1002600050E0C8E7D0E014C0C19A8F2D902F04C091
:10027000FD013197F1F701970097D1F7C198CB01B4
:1002800004C0FD013197F1F701970097D1F72F5F77
:100290002E1550F39A0109C080E197E2FE013197D3
:1002A000F1F70197D9F72150304021153105A1F719
:1002B00020E0EECFB99AC19891E29FBD91E093BF43
:1002C000880F880F90E049965FD012BE89BDFFCF9E
:1002D0001F9380E69AEE0197F1F780E090E054D00A
:1002E00080936D00682F6F5F6A3008F060E080E0F7
:1002F00090E052D08FEF87BB18BA87E0A5DE10914F
:100300006D00812F880F880F90E048963DD0E82F30
:10031000F0E0EE0FFF1FE05AFF4F0190F081E02D5B
:10032000812F0995FFCF1F920F920FB60F921124C4
:100330002F933F934F935F936F937F938F939F93ED
:10034000AF93BF93EF93FF9380916A00882359F096
:1003500010926A0080E090E060916D001DD081E015
:1003600090E060E019D0FF91EF91BF91AF919F9124
:100370008F917F916F915F914F913F912F910F904E
:100380000FBE0F901F901895E199FECF1FBA8EBB3C
:10039000E09A99278DB30895262FE199FECF1CBAD4
:1003A0001FBA8EBB2DBB0FB6F894E29AE19A0FBE2E
:0803B00001960895F894FFCFB7
:0C03B8005A014C001101A200D00001000D
:00000001FF
